:0200000080740A
:06000B00C2AFC28C80535D
:10001B00C2AFC28EC0D0C0E0758DFF758BFFE530CF
:10002B002401D4B4601B753000E5312401D4B460D5
:10003B0014753100E5322401D4B4240D75320080DF
:10004B000AF5308006F5318002F532BD0002053726
:10005B00D0E0D0D0D2AFD28E320F0E000000000015
:10006B00758A8A758CECD2AFD28C32C2B0C2B1D247
:10007B00B2C290C2917581507F007E007D007520C9
:10008B0000753000753100753200758A8A758CECFD
:10009B00758BFF758DFF758951D2A9D2ABD2AFD2BB
:1000AB008CD28E20B702516F519F516311C33129EE
:1000BB00318631CC514580F4EDB40416740075F0E3
:1000CB00EC3161740175F0EC3161740275F0E6315D
:1000DB006122E530540FF8E530C4540F75F00AA4D3
:1000EB002875F004A4F5F074003161E531540FF874
:1000FB00E531C4540F75F00AA42875F004A4F5F08B
:10010B0074013161E532540FF8E532C4540F75F0C8
:10011B000AA42875F00AA4F5F07402316122ED707F
:10012B0005C290C29122B40105D290C29122B402B1
:10013B0005C290D29122B40305D290D2912274328F
:10014B00C39F50117F0074035C70027401FC139207
:10015B00901392910C225407234400C478043176F7
:10016B00E5F078083176C2B2D2B222334004C2B085
:10017B008002D2B0D2B1C2B1D8F122309242200665
:10018B003F20073CED6039309310300409EE24FC1E
:10019B00502EC204802AC205802630050BEE24CDDA
:1001AB00501E7E00510F8018300411EE24FD5010AC
:1001BB00D205C2047E00D203510F8004D2047E000C
:1001CB0022309210300609EE24FC5037C2068033E1
:1001DB00C207802F30070FEE24CD50277E000DBDB8
:1001EB0005217D00801D300616EE24FD5015D2072B
:1001FB00C2067E007537000DBD05087D008004D258
:10020B00067E0022EDB40103512722B402035134C0
:10021B0022B403035141227F007C0122E5322401E9
:10022B00D4B424027400F53222E5312401D4B46035
:10023B00027400F531227530002230031AE537C302
:10024B00940A4013C20385302285312385322475ED
:10025B002C00752D0051C622E52AB4AA07E52BB454
:10026B00550280267522007523007524007525071D
:10027B00752601752701752805752910752AAA752C
:10028B002B55752C00752D0051C6852230852331D9
:10029B0085243222712574D051E4701E740051E410
:1002AB007018712E712574D0D2E051E4700C782245
:1002BB00790C51FD08D9FB712E2222712574D05176
:1002CB00E47015740051E4700F7822790CE651E458
:1002DB00700608D9F8712E22227A0820E704C2B4DE
:1002EB008002D2B47156713B23DAF0D2B4715671DD
:1002FB004422D2B474007A08C0E071446007D0E0A5
:10030B00D2E0238003D0E023DAEE03F6B90104D266
:10031B00B48002C2B47156713B22C2B47156C2B3DF
:10032B00715622C2B47156D2B37156D2B4715622E1
:10033B00D2B37156C2B3715622D2B3715620B404E4
:0D034B00740080027401C2B37156220022BA
:00000001FF
